:100000000C942A000C9447000C9447000C94470071
:100010000C947C050C9447000C9447000C9447000A
:100020000C9447000C9447000C9447000C94470034
:100030000C9447000C9447000C9447000C94470024
:100040000C9447000C9447000C9447000C94470014
:100050000C94470011241FBECFE5D8E0DEBFCDBF12
:1000600010E0A0E6B0E0E2EAF1E102C005900D92F6
:10007000A636B107D9F712E0A6E6B0E001C01D929E
:10008000AD39B107E1F70E948E020C94CF080C94B1
:100090000000EF92FF920F931F930E942104939808
:1000A00085E40E945604939A85E88A95F1F793981F
:1000B00080E00E945604E82EFF2400E010E0102F9C
:1000C0000F2DFE2CEE2480E00E94560490E0A0E06C
:1000D000B0E0E82AF92A0A2B1B2B102F0F2DFE2C3B
:1000E000EE2480E00E945604939A282F30E040E0EE
:1000F00050E02E293F29402B512BB901CA011F91F5
:100100000F91FF90EF9008950E942104939881E051
:100110000E945604939A939881E00E945604939A01
:1001200008951F93182F0E942104939881E00E9444
:100130005604939A9398112311F082E001C083E052
:100140000E945604939A1F9108951F930E942104C0
:100150009798979A939884E40E945604939A15E886
:10016000812F8A95F1F7939880E00E945604939A24
:10017000812F8A95F1F7939887E00E945604939A0D
:10018000812F8A95F1F7939883E00E945604939A01
:10019000812F8A95F1F7939880E00E945604939AF4
:1001A000812F8A95F1F7939884E00E945604939AE0
:1001B000812F8A95F1F7939882E50E945604939ACD
:1001C000812F8A95F1F7939883E00E945604939AC1
:1001D000812F8A95F1F7939881E30E945604939AB0
:1001E000812F8A95F1F7939882E00E945604939AA2
:1001F000812F8A95F1F793988EE80E945604939A7E
:10020000812F8A95F1F7939881E00E945604939A82
:10021000812F8A95F1F7939883E00E945604939A70
:10022000812F8A95F1F7939884E40E945604939A5B
:10023000812F8A95F1F7939880E00E945604939A53
:100240001A95F1F71F91089584B780934C0214BE5C
:100250008898899ABA9ABB9AD798A798D6988AB359
:100260008F638ABB84B38F6784BBBC9A8B9A8C9A4A
:100270008D9AC49A939A949A959ABD9ABF9ABE9869
:10028000C59AC79A8E988F9A8A9808952FB78D5FCE
:10029000F894A89591B5986191BD81BD2FBF08953F
:1002A000EF92FF920F931F93CF93DF93E82E8B0172
:1002B000F42E41E0C82FD0E01AC0CE01840F911D6A
:1002C0006F2D70E00E94BC08382F86958695869524
:1002D000F801E80FF11D808190E0232F277002C004
:1002E000959587952A95E2F780FD04C04F5FF41637
:1002F00020F73E2D832FDF91CF911F910F91FF901B
:10030000EF90089564E770E040E40E945001089582
:100310006AE871E044E50E9450010895CF93DF93AD
:10032000EC01DB0120E030E00DC08D918095FE01F5
:10033000E20FF31F908189232F5F3F4F882311F035
:1003400080E003C0241788F381E0DF91CF91089506
:100350006AE871E0CB01655F7F4F4BE00E948E0140
:1003600080934B02089564E770E0CB01685F7F4F94
:1003700048E00E948E0180934A0208950E94A801DD
:10038000882319F480E090E008950E94B30190E082
:10039000882309F491E081E09827892F0895E5E901
:1003A000F1E0119281E0E03AF807D9F70895E0EA28
:1003B000F1E01192119282E0E834F807D1F7089544
:1003C000ECE7F0E0119280E0E438F807D9F70895FF
:1003D000E4E8F0E0119211921192119281E0E43878
:1003E000F807C1F70895ECE7F0E0119280E0E438F7
:1003F000F807D9F7E5E9F1E0119281E0E03AF80772
:10040000D9F708950F931F93CF93DF938C014FEF8C
:1004100050E0EFEFF0E020C0DB016531710510F036
:10042000A4E1B0E09D01E8018991480F511DE40F5E
:10043000F51F21503040C1F70A0F1B1F6A1B7B0BB1
:10044000852F99279C01240F311DA9018F2F9927F2
:100450009C012E0F311DF90161157105E9F6852FFB
:1004600099272F2F33272E0F311D322F2227840F4C
:10047000911D282B392BC901DF91CF911F910F912D
:1004800008950F931F93CF93DF9384E890E060E08B
:1004900071E00E940202909385018093840180EABA
:1004A00091E068EA70E00E94020290934902809312
:1004B0004802CEEDD1E000E010E0C80182599F4F24
:1004C000BE010E940D07C81BD90B080F191F2097EA
:1004D000A1F7C7E0D0E000E010E0C801845B9D4FC9
:1004E000BE010E940D07C81BD90B080F191F2097CA
:1004F000A1F7DF91CF911F910F91089586B186608A
:1005000086B93098359A80B78F7180BF379A3E98F8
:100510003F9887B1866087B9369A0895CF92DF9267
:10052000EF92FF920F931F93CF93DF9310924A02A3
:1005300010924B02E4E7F0E08FEF80831086319653
:1005400020E0EC37F207C9F7EAE8F1E080E02FE0BD
:100550009FEF8A3011F0908302C02093940113869C
:100560008F5F31968B30A9F70E9424010E941504F9
:100570000E9471050E947E020E94B8050E94FF073A
:100580000E94A500789411E0E12EF12CB0E2CB2E70
:10059000BEE4DB2E0E9489088091510290915202A4
:1005A00069E170E00E94A808892B91F480916B00AA
:1005B000882371F00E94F005EC01009749F00E9439
:1005C000F005C817D90721F00E94F005EC01F7CF1C
:1005D0000E94BE01882341F00E9441020E94E00176
:1005E0000E94CF010E94D701349B53C080914B02DF
:1005F000882309F04EC094B185B1349A182F00E0D9
:10060000692F70E0602B712B7093890160938801D2
:1006100020918601283269F580918701482F50E0AA
:10062000FA01EE0FFF1FE056FE4F20813181620F6D
:10063000731F71836083E82FE695E695E695F0E0F9
:10064000EB56FE4F47705070970102C0220F331FC8
:100650004A95E2F79081922B90830E9488018093C3
:1006600087010E948E0310928601C6010197F1F75F
:1006700010C0E0918701F0E0EE0FFF1FE056FE4F43
:1006800080819181680F791F718360832F5F209330
:10069000860186997FCF80914A02882309F07ACF1C
:1006A0000E944900AB01BC0140937000509371005F
:1006B000609372007093730080916E00823051F5E8
:1006C00080916F00282F30E0F901EE0FFF1FEE0F31
:1006D000FF1FE259FF4F468B578B608F718F10922F
:1006E0006E00E82FE695E695E695F0E0E259FF4FBB
:1006F00027703070A70102C0440F551F2A95E2F7FA
:100700009685942B96870E94820180936F000E94A9
:10071000C20340CF8F5F80936E003CCF883248F495
:10072000282F30E0843210F02F5F3F4F922F990F27
:1007300023C0803560F48852282F30E0843210F0D6
:100740002F5F3F4F220F331F922F9F5F15C08435BD
:1007500090F48055813049F0813028F0823039F0B2
:10076000833049F406C098E407C099E405C092E5D7
:1007700003C093E501C090E085B39F778078982B04
:1007800095BB0895282F82958F70823041F0833079
:1007900041F0882311F490E105C090E003C090E39C
:1007A00001C090E28BB32F70922B807C982B9BBB67
:1007B00008951DB88091670280FF02C06D9A01C044
:1007C0006D988DB18091540280FF02C06B9A01C078
:1007D0006B988DB18091650280FF02C06A9A01C05A
:1007E0006A988DB180916602833091F0843028F44C
:1007F000813051F0823050F410C0853089F085305E
:1008000048F0863051F407C0699A0AC0699A03C05B
:10081000689A06C0689A709A04C08DB183608DB9D9
:1008200070988DB180658DB9089584E080936602DB
:100830001092670210925402109265020E94D9032E
:10084000089586E0809366021092670281E08093AB
:100850005402809365020E94D903089510926602A3
:100860001092670210925402109265020E94D903FE
:100870000895873008F086E0809366020E94D903CD
:100880000895811181E0809367020E94D903089541
:10089000811181E0809354020E94D903089581114F
:1008A00081E0809365020E94D90308956C9B6C9A45
:1008B0008FB9779BFECF8FB10895AF92BF92CF9241
:1008C000DF92EF92FF920F931F93CF93DF93C82E87
:1008D000D62EEE24FF24862F90E026E6A22E20E0DE
:1008E000B22EA80EB91EEC01C05ADF4F01E010E095
:1008F0007FC0C39AF50180818823C1F0DD2059F4BF
:1009000028B38881A80102C0440F551F8A95E2F7D9
:10091000242B28BB26C022B38881F80102C0EE0F29
:10092000FF1F8A95E2F72E2B22BB1BC0DD2069F446
:1009300028B38881A80102C0440F551F8A95E2F7A9
:10094000CA018095822388BB0CC022B38881F8013C
:1009500002C0EE0FFF1F8A95E2F7CF018095822338
:1009600082BBC398F701EB5AFD4F80810E94560469
:10097000F701E859FD4F8083C39AF50180818823F0
:10098000E1F0DD2069F428B38881A80102C0440F9A
:10099000551F8A95E2F7CA018095822388BB24C03F
:1009A00022B38881F80102C0EE0FFF1F8A95E2F79B
:1009B000CF018095822382BB17C0DD2059F428B374
:1009C0008881A80102C0440F551F8A95E2F7242BA5
:1009D00028BB0AC022B38881F80102C0EE0FFF1FB6
:1009E0008A95E2F72E2B22BBC3980894E11CF11CD8
:1009F000EC1408F47ECFDF91CF911F910F91FF90FF
:100A0000EF90DF90CF90BF90AF900895FF920F933B
:100A10001F93CF93DF93F82E042F442379F488B3E8
:100A20009091600021E030E002C0220F331F9A95C0
:100A3000E2F7822788BBEB0110E014C022B3E42F59
:100A4000F0E0E05AFF4F308181E090E002C0880F73
:100A5000991F3A95E2F7282722BBEDCF89910E9492
:100A600056041F5F1F15D0F3002369F488B39091DB
:100A7000600021E030E002C0220F331F9A95E2F7B8
:100A8000822788BB0FC022B3E02FF0E0E05AFF4F6F
:100A9000308181E090E002C0880F991F3A95E2F71B
:100AA000282722BBDF91CF911F910F91FF900895CE
:100AB000982F6C9A20E030E011C0C498F901EB5AED
:100AC000FD4F80818FB9F901E859FD4F02C08FB108
:100AD0008083779BFCCFC49A2F5F3F4F291768F321
:100AE000089588E085BD85B5836085BD8CE783BDAD
:100AF00089B7806889BF08951F920F920FB60F9231
:100B000011242F938F939F93AF93BF9380915102A2
:100B100090915202875E934050F4809151029091DF
:100B200052020196909352028093510217C0109284
:100B300052021092510280914D0290914E02A0916A
:100B40004F02B09150020196A11DB11D80934D023C
:100B500090934E02A0934F02B0935002BF91AF9179
:100B60009F918F912F910F900FBE0F901F9018950E
:100B7000C29884EF91E028EC30E0F9013197F1F769
:100B80000197D9F7C29A80E197E20197F1F70895AA
:100B90000F931F938C010E942E048FE080935502C7
:100BA00010935602009357021092580284E00E945C
:100BB000580580916B021F910F9108950F931F9319
:100BC00088E294E00E94C805182F00E089E294E0D2
:100BD0000E94C805080F111DC8011F910F910895AB
:100BE0001F9386E294E00E94C805182F87E294E0E4
:100BF0000E94C805512F40E0282F30E0242B352BD0
:100C0000C9011F9108950F931F9384E294E00E94FD
:100C1000C805182F00E085E294E00E94C805080F7F
:100C2000111DC8011F910F9108950F931F9382E228
:100C300094E00E94C805182F00E083E294E00E942F
:100C4000C805080F111DC8011F910F9108950F933A
:100C50001F9380E294E00E94C805182F00E081E213
:100C600094E00E94C805080F111DC8011F910F9143
:100C7000089583E094E00E94C805089583E094E01D
:100C80000E94C805873121F481E080936A0002C088
:100C900010926A0080916A000895FF920F931F934B
:100CA000F82E192F062F0E942E0480EF80935502F4
:100CB00010935602F09257020093580284E00E946B
:100CC00058051F910F91FF9008951F93182F692FBA
:100CD00088E294E00E944D0689E294E0612F0E9430
:100CE0004D061F9108954F925F926F927F928F925F
:100CF0009F92BF92CF92DF92EF92FF920F931F933A
:100D0000CF93DF93082F0E94F0059C01009711F408
:100D1000BB2464C0B02E44E0401710F444E0B42E6D
:100D20008B2D90E02817390708F4B22E0E94DE05BB
:100D30002C019C013F70C12C90E6D92EC20ED31E0F
:100D40008B2C9924C401820F931F8150904118F479
:100D5000C0E0D0E037C0E12C80E1F82EE21AF30ABF
:100D600034016E187F0800E009C0CE018C0D9D1D76
:100D70000E94C805C758DD4F88830F5FC02FD0E0A1
:100D8000CE15DF0590F3DD240CC08C010E0D1F1D68
:100D90008050904A0E94C80507581D4FF801808373
:100DA000D3948D2D90E08615970578F30DC0C6017C
:100DB0000E94C805FE01E758FD4F808321960894E4
:100DC000C11CD11CCB1598F3C401840D951D0E9444
:100DD000650681E094E060E40E944D068B2DDF9172
:100DE000CF911F910F91FF90EF90DF90CF90BF9028
:100DF0009F908F907F906F905F904F9008951F937A
:100E0000182F692F84E294E00E944D0685E294E059
:100E1000612F0E944D061F9108956F927F928F92CD
:100E20009F92AF92BF92CF92DF92EF92FF920F9379
:100E30001F93CF93DF934C016B010E942706EC01B7
:100E400010E00E942706C817D90721F00E94270644
:100E5000EC0101C01F5F1330A0F3209719F4CC24DC
:100E6000DD2465C00E9403065C0110E00E940306B9
:100E7000A816B90621F00E9403065C0101C01F5F9D
:100E80001330A0F395013F70E12C50E4F52EE20EF3
:100E9000F31ECC15DD0508F46E01C601820F931F09
:100EA0008150904118F4C0E0D0E034C000E010E17F
:100EB000021B130B3601601A710AC0E0D0E0F40186
:100EC000EC0FFD1FC70160810E944D06219608941A
:100ED000E11CF11CC017D10790F3080D191DC0E0EB
:100EE000D0E009C0CE018050904AF80161918F0195
:100EF0000E944D062196C615D705A0F30EC0F40139
:100F0000EC0FFD1FC70160810E944D0621960894D9
:100F1000E11CF11CCC15DD0590F3C6018A0D9B1D6B
:100F20000E94FF0681E094E060E20E944D06C60147
:100F3000DF91CF911F910F91FF90EF90DF90CF90B5
:100F4000BF90AF909F908F907F906F9008959091F9
:100F50007802903248F4E92FF0E0E358FD4F8AE040
:100F600080839F5F90937802609178028DE792E092
:100F700070E00E940D07109278020895DC010BC00A
:100F80009032F0F7E92FF0E0E358FD4F80839F5F48
:100F90009093780211968C9190917802882381F732
:100FA000903248F4E92FF0E0E358FD4F8AE0808367
:100FB0009F5F90937802609178028DE792E070E0F5
:100FC0000E940D07109278020895DC010BC0603278
:100FD000F0F7E62FF0E0E358FD4F80836F5F6093FA
:100FE000780211968C9160917802882381F78DE7C1
:100FF00092E070E00E940D0710927802089589E057
:1010000090E06AEF0E944D068AE090E067EC0E9453
:101010004D068BE090E06FE00E944D068CE090E082
:101020006DEA0E944D068DE090E062E20E944D065E
:101030008EE090E061E00E944D068FE090E06AE073
:101040000E944D0680E190E060E00E944D0681E143
:1010500090E060E80E944D0682E190E06FE70E9418
:101060004D0685E090E06FEF0E944D0686E090E02F
:101070006FEF0E944D0687E090E06FEF0E944D06F3
:1010800088E090E060E00E944D0681E090E06AE038
:101090000E944D0682E090E060E00E944D0683E0F1
:1010A00090E060E00E944D0684E090E060E00E94E5
:1010B0004D068AE190E06AE00E944D068BE190E0E7
:1010C0006AE00E944D0680E094E061E00E944D06D7
:1010D00084E094E063E10E944D0685E094E068E8D6
:1010E0000E944D0681E094E061E00E944D0683E09D
:1010F00094E00E94C8058331D1F781E094E062E07A
:101100000E944D0683E094E00E94C8058431D1F727
:1011100008951F930E943906182F873139F08431C2
:1011200059F00E943906182F873121F481E080930D
:101130006B000BC0843119F410926B0006C0109242
:101140006B000E94B8050E94FF07812F1F91089530
:10115000AA1BBB1B51E107C0AA1FBB1FA617B707DD
:1011600010F0A61BB70B881F991F5A95A9F78095F9
:101170009095BC01CD01089597FB092E07260AD052
:1011800077FD04D0E5DF06D000201AF47095619554
:101190007F4F0895F6F7909581959F4F0895F894A5
:0211A000FFCF7F
:0611A20004030405010036
:00000001FF
